:1000000000308A00DF280000B9010408B800391068
:10001000831B3914B21F1428B817381EB80AB10947
:10002000B209B10A0319B20A320EF038B400B407AB
:10003000E23EB500323EB70032080F39B507B507CA
:10004000B707E93EB600B607B607310E0F39B60757
:10005000B707B60DB70DB709B70D31080F39B70798
:10006000B40D0730B3000A30B707B603031C3428B9
:10007000B607B503031C3828B507B403031C3C2896
:10008000B407B303031C40283330840083130730C4
:100090003805381384033805031D5528381A840A97
:1000A000381A55282030F7007228840737300402A8
:1000B000031938170008F700031D6628381B662847
:1000C000381A7628B819662820307128B81F6E288B
:1000D0002D30F70084033813B8137228B81538127E
:1000E0003030F70777080C1E73289900840A381FF0
:1000F000562800340B0884008B13E03003178D055D
:1001000083168C170C152630840083132030F700DB
:100110000C140000000083120D087A0203199728BE
:100120000C088000840A0E088000840A9D28780844
:100130008000840A79088000840A8D0AF70BA128C0
:10014000A328831688288D03E0308D05263084008F
:1001500083132030F70000088C00840A00088E000A
:10016000840A553083168D00AA308D008C1400004F
:1001700000000000000083128D0AF70BAB288316E5
:100180000C110408831203138B048A110A12242A07
:1001900027308400831300080319DC280130F8009D
:1001A000F701F70BD128F80BD0284A30F700F70BEE
:1001B000D728DA28800BCE288A110A12322A840125
:1001C00083131F3083058316031787111930031318
:1001D0009900A63098009030831298008316031778
:1001E0000908C039890003131F129F12003003173A
:1001F00088008312870188018901FF300313A00062
:10020000A1010530A200831603170908C03989002F
:1002100003131F129F120F3003178800831203135A
:100220001F179F1783169F1783121F149412A01273
:100230002008831687008312201620088316870063
:100240008312A011200883168700013083129400C6
:100250000030831694000108C739083881008312E2
:1002600090010030F8009200003083169200831253
:10027000031787018801890183160313061083126F
:100280000610831605168312051AF72983168610A1
:10029000831286140530A200A10122081F3C031C12
:1002A000F129031D57292108FE3C031CF1292108CF
:1002B00003178D000313220803178F0083168C1772
:1002C0000C140000000083120E08FA000C0803133F
:1002D000A6007A08A70001302107A8002208A9007B
:1002E0000318A90A280803178D0003132908031708
:1002F0008F0083168C170C140000000083120E0868
:10030000FA000C080313A9007A08AA00023021079A
:10031000AB002208AC000318AC0A2B0803178D00B1
:1003200003132C0803178F0083168C170C1400007E
:10033000000083120E08FA000C080313AC007A08C0
:10034000AD0003302107AE002208AF000318AF0A4A
:100350002E0803178D0003132F0803178F00831631
:100360008C170C140000000083120E08FA000C0811
:100370000313AF007A08B000103084002708B200E1
:100380002608B10004202C300C1EC429990010301E
:1003900084002A08B2002908B10004202C300C1E69
:1003A000CF299900103084002D08B2002C08B1002C
:1003B00004202C300C1EDA299900103084003008FB
:1003C000B2002F08B10004200A300C1EE529990064
:1003D0000D300C1EE92999000430A1070318A20A68
:1003E0004D298316861083128610F529362A220895
:1003F0001F3C031C352AA3012308033C031C292AA4
:10040000230DF700F70DFC30F7051F08C3397704FB
:100410009F000330F700F70B0B2A9F149F180E2A3A
:1004200083161E088312A4001E08A50021080317C6
:100430008D00FA000313220803178F00031324080A
:10044000F8002508F9007A28A10A0319A20AA30ACC
:10045000FC2983168610023083128606A600E1303E
:0E046000A700C828A60B2F2AF729352A63000B
:04400E00C12FFF3F80
:00000001FF
